:1000000009C021C020C020C01EC01DC01CC01BC014
:100010001AC019C011241FBECFE9CDBF10E0A0E661
:10002000B0E0E4EDF3E002C005900D92A236B10716
:10003000D9F720E0A2E6B0E001C01D92A137B207D7
:10004000E1F7B4D0C5C1DCCF1F920F920FB60F926B
:1000500011242F933F934F935F936F937F938F93CD
:100060009F93AF93BF93EF93FF9380916F00909115
:10007000700001969093700080936F002091600053
:10008000309161002817390708F057C080E891E0E7
:1000900090936100809360001092700010926F0046
:1000A000369A3699FECF85B18093680080916800BA
:1000B0008639E8F481E08093630082E080936500F4
:1000C0006091630088E090E072D16091650080E10A
:1000D00090E06DD188B3837E88BB2FE789EA93E0F7
:1000E000215080409040E1F700C0000026C0809180
:1000F0006800803B30F4809163008F5F80936300E1
:100100000FC080916300853010F0109263008091E1
:100110006800823D60F4809165008F5F8093650088
:1001200080E093E0909361008093600006C080912E
:100130006500853010F010926500FF91EF91BF913E
:10014000AF919F918F917F916F915F914F913F916F
:100150002F910F900FBE0F901F9018958091620005
:10016000813069F040F0823079F0833099F4C29A9E
:1001700088B3877E0EC0C49A88B3837F0AC088B3D1
:10018000886188BBC29806C088B38C6088BBC4985D
:1001900001C088BB809162008F5F80936200809174
:1001A0006200843010F010926200089587B38F616E
:1001B00087BB83B7816083BF8FB583608FBD8FB5E9
:1001C000806E8FBD8FE786BF89BD89B7826089BF8A
:1001D00078943D9A86B1846886B988E090E0E0D052
:1001E0008093630080E190E0DBD080936500809194
:1001F0006300853018F081E0809363008091650092
:10020000853018F082E0809365008DE0382E9AE00A
:10021000492E28E0722E38E2632E44E1542EC0EAC3
:10022000DFE008EB1BE050E6E52E59E0F52E60EE2E
:10023000C62E6EE2D62E70E7A72E77E1B72EE9E044
:100240008E2E912C80916300823091F038F48823B7
:1002500061F0813091F4509267000FC0833059F003
:10026000843059F47092670008C06092670005C03E
:100270003092670002C04092670080916A009091BE
:100280006700890F80936A0080916A00853670F15B
:10029000909163008091640098130CC09091650068
:1002A00080916E00981306C0809169008F5F8093E3
:1002B000690002C010926900809169008A3061F47F
:1002C0006091630088E090E072D06091650080E109
:1002D00090E06DD01092690080916300809364007B
:1002E0008091650080936E0010926A008091650095
:1002F000880F80936D00809163008230C1F048F4D4
:10030000882381F08130E1F4B0926C00A0926B0000
:1003100017C0833089F0843099F4F0926C00E09239
:100320006B000EC0D0926C00C0926B0009C0D093DD
:100330006C00C0936B0004C010936C0000936B00C2
:100340000DDF109266009091660080916D00891714
:1003500060F080916B0090916C000197F1F78091B3
:1003600066008F5F80936600EECFF8DE1092660025
:100370008091660020916D0090E0A401421B51091C
:10038000841795070CF05ECF80916B0090916C0004
:100390000197F1F7809166008F5F80936600E8CF48
:1003A000E199FECF8EBBE09A99278DB30895262F51
:1003B000E199FECF8EBBE09A81500DB2021639F062
:1003C0001CBA2DBB0FB6F894E29AE19A0FBE0895BD
:0403D000F894FFCFCF
:0203D4008001A6
:00000001FF
